:020000040000FA
:04080000D8EF07F036
:1008100003B213EF05F0F2B431EF05F09EB039EFFB
:1008200005F09EB241EF05F0F2A81AEF04F0F2B223
:1008300025EF04F0F2A620EF04F0F2B022EF04F06E
:1008400087EF07F0F296F290FF00CD90F2929EA013
:100850002FEF04F00101533F2FEF04F0542BAEC1F2
:10086000B2F1AFC1B3F1B0C1B4F1B1C1B5F1AAC138
:10087000AEF1ABC1AFF1ACC1B0F1ADC1B1F1A6C148
:10088000AAF1A7C1ABF1A8C1ACF1A9C1ADF1A2C158
:10089000A6F1A3C1A7F1A4C1A8F1A5C1A9F19EC168
:1008A000A2F19FC1A3F1A0C1A4F1A1C1A5F19AC178
:1008B0009EF19BC19FF19CC1A0F19DC1A1F196C188
:1008C0009AF197C19BF198C19CF199C19DF1CECF4E
:1008D00096F1CFCF97F153C198F154C199F1CF6AF6
:1008E000CE6A0101536B546B9E90CD800FBC0F8E6E
:1008F0000FBA7EEF04F00F8A87EF07F00F8C0FBE60
:10090000BAEF04F096C19AF197C19BF198C19CF19E
:1009100099C19DF19AC19EF19BC19FF19CC1A0F12B
:100920009DC1A1F19EC1A2F19FC1A3F1A0C1A4F1FB
:10093000A1C1A5F1A2C1A6F1A3C1A7F1A4C1A8F1CB
:10094000A5C1A9F1A6C1AAF1A7C1ABF1A8C1ACF19B
:10095000A9C1ADF1AAC1AEF1ABC1AFF1ACC1B0F16B
:10096000ADC1B1F1AEC1B2F1AFC1B3F1B0C1B4F13B
:10097000B1C1B5F101015E6B5F6B606B616B96514C
:100980005E2797515F2398516023995161239A51B3
:100990005E279B515F239C5160239D5161239E5193
:1009A0005E279F515F23A0516023A1516123A25173
:1009B0005E27A3515F23A4516023A5516123A65153
:1009C0005E27A7515F23A8516023A9516123AA5133
:1009D0005E27AB515F23AC516023AD516123AE5113
:1009E0005E27AF515F23B0516023B1516123B251F3
:1009F0005E27B3515F23B4516023B5516123D89072
:100A00000101613360335F335E33D890010161339C
:100A100060335F335E33D8900101613360335F33FD
:100A20005E3387EF07F00392ABB2AB98AB8803015C
:100A300003EE00F080517F0BE92604C0EFFF802B0E
:100A40008151805D700BD8A48B8200008051815D44
:100A5000700BD8A48B9281518019D8B4079087EF7E
:100A600007F0F2940101453F87EF07F0462B87EF2F
:100A700007F09E900101533F87EF07F0542B87EF5B
:100A800007F09E92040062A146EF05F0077C07ACD8
:100A900061EF05F0C274C2B45BEF05F0C3CFB3F5EC
:100AA000C4CFB4F50501D890B433B333D890B43380
:100AB000B33362EF05F0C3CF55F1C4CF56F162EF07
:100AC00005F0C28207B4CFEF05F047C14BF148C132
:100AD0004CF149C14DF14AC14EF15EC162F15FC1B5
:100AE00063F160C164F161C165F196C1B6F197C16E
:100AF000B7F198C1B8F199C1B9F19AC1BAF19BC1E6
:100B0000BBF19CC1BCF19DC1BDF19EC1BEF19FC1B5
:100B1000BFF1A0C1C0F1A1C1C1F1A2C1C2F1A3C185
:100B2000C3F1A4C1C4F1A5C1C5F1A6C1C6F1A7C155
:100B3000C7F1A8C1C8F1A9C1C9F1AAC1CAF1ABC125
:100B4000CBF1ACC1CCF1ADC1CDF1AEC1CEF1AFC1F5
:100B5000CFF1B0C1D0F1B1C1D1F1B2C1D2F1B3C1C5
:100B6000D3F1B4C1D4F1B5C1D5F1B3C5B5F5B4C5B0
:100B7000B6F5B5C5B7F5B6C5B8F5010155515B2752
:100B800056515C23E86A5D230E2ECFEF05F05CC161
:100B900057F15DC158F15B6B5C6B5D6B078E0201B9
:100BA000002F87EF07F03C0E006F05012F51000A60
:100BB000D8B486EF06F005012F51010AD8B410EF22
:100BC00006F005012F51020AD8B451EF06F00501D5
:100BD0002F51030AD8B451EF06F005012F51040A32
:100BE000D8B451EF06F005012F51050AD8B451EFE2
:100BF00006F005012F51060AD8B451EF06F00501A1
:100C00002F51070AD8B451EF06F005012F51320ACF
:100C1000D8B40EEF06F02F6B86EF06F086EF06F0E5
:100C2000050153671BEF06F054671BEF06F055678D
:100C30001BEF06F056671FEF06F086EF06F057C56C
:100C400000F158C501F159C502F15AC503F101017E
:100C5000010E046F000E056F000E066F000E076F89
:100C600081EC1EF000C157F501C158F502C159F5DC
:100C700003C15AF5006744EF06F0016744EF06F040
:100C8000026744EF06F0036786EF06F053C557F599
:100C900054C558F555C559F556C55AF50F8886EF10
:100CA00006F00501306757EF06F086EF06F00FBE3D
:100CB0006CEF06F010A071EF06F00101476768EFD6
:100CC00006F0486768EF06F0496768EF06F04A6784
:100CD0006CEF06F071EF06F007AE71EF06F083EFF0
:100CE00006F00501312F86EF06F03C0E316F302FF4
:100CF00086EF06F00101000E626FE00E636FA50E35
:100D0000646F010E656F0501306B0F880501626B22
:100D100033B78CEF06F062810CC100F10DC101F117
:100D20000EC102F10FC103F110C104F111C105F1AF
:100D300012C106F113C107F114C108F115C109F17F
:100D400016C10AF117C10BF135C134F100C10CF124
:100D500001C10DF102C10EF103C10FF104C110F187
:100D600005C111F106C112F107C113F108C114F157
:100D700009C115F10AC116F10BC117F134C135F1E2
:100D800001018A67CBEF06F08B67CBEF06F08C672B
:100D9000CBEF06F08D67CFEF06F0FFEF06F08EC1C8
:100DA00000F18FC101F190C102F191C103F1010184
:100DB000010E046F000E056F000E066F000E076F28
:100DC00081EC1EF000C18EF101C18FF102C190F1E2
:100DD00003C191F10067F4EF06F00167F4EF06F04C
:100DE0000267F4EF06F00367FFEF06F08AC18EF1A9
:100DF0008BC18FF18CC190F18DC191F10F80D57EA7
:100E0000D5BE69D0D6CF47F1D7CF48F145C149F11A
:100E1000E86AE8CF4AF1109047C100F148C101F1FA
:100E200049C102F14AC103F101010A0E046F000E2B
:100E3000056F000E066F000E076F81EC1EF003AF0A
:100E40001080010154A731EF07F00F9A0F9C0F9EFD
:100E50000101000E5E6F600E5F6F3D0E606F080E49
:100E6000616F010147BF41EF07F0486741EF07F0AD
:100E7000496741EF07F04A6741EF07F0F28866EFF4
:100E800007F0F2985E6B5F6B606B616B966B976BB4
:100E9000986B996B9A6B9B6B9C6B9D6B9E6B9F6B1E
:100EA000A06BA16BA26BA36BA46BA56BA66BA76BCE
:100EB000A86BA96BAA6BAB6BAC6BAD6BAE6BAF6B7E
:100EC000B06BB16BB26BB36BB46BB56BD76AD66AF0
:100ED0000101456B466B0CC100F10DC101F10EC162
:100EE00002F10FC103F110C104F111C105F112C1EA
:100EF00006F113C107F114C108F115C109F116C1BA
:100F00000AF117C10BF135C134F187EF07F002C0C8
:100F1000E0FF005001C0D8FF1000A6B28DEF07F02F
:100F20000CC0A9FF0BC0A8FFA69EA69CA684F29E9B
:100F3000550EA76EAA0EA76EA682F28EA694A6B232
:100F40009FEF07F00C2A1200A96EA69EA69CA68011
:100F5000A8500C2A120004012C0E826F92EC0AF0A9
:100F60007CEC1FF00C50A4EC07F0E8CF00F10C5023
:100F7000A4EC07F0E8CF01F101AFC4EF07F00101E5
:100F8000FF0E026FFF0E036F1FEC1FF02967D0EFFB
:100F900007F00401200E826F92EC0AF0D5EF07F003
:100FA00004012D0E826F92EC0AF049EC1DF0120044
:100FB000076A0F6A106A0F010D0EC16E860EC06EB1
:100FC000030EC26E0F01680E896E130E926E080E2C
:100FD0008A6EF30E936E8B6A900E946EF18EF19E74
:100FE0000E6A01015B6B5C6B5D6B576B586BF29A21
:100FF0000101476B486B496B4A6B4B6B4C6B4D6BFC
:101000004E6B4F6B506B516B526B456B466BD76A97
:10101000D66A0F01280ED56EF28A9D90B00ECD6E65
:1010200001015E6B5F6B606B616B626B636B646B2A
:10103000656B666B676B686B696B536B546BCF6AE0
:10104000CE6A0F9A0F9C0F9E9D80760ECA6E9D826F
:1010500002013C0E006FCC6A160EA4EC07F0E8CF3C
:1010600000F1170EA4EC07F0E8CF01F1180EA4EC84
:1010700007F0E8CF02F1190EA4EC07F0E8CF03F176
:10108000010103AF5EEF08F07CEC1FF0160E0C6E52
:1010900000C10BF08DEC07F0170E0C6E01C10BF0C8
:1010A0008DEC07F0180E0C6E02C10BF08DEC07F002
:1010B000190E0C6E03C10BF08DEC07F000C18AF124
:1010C00001C18BF102C18CF103C18DF100C18EF120
:1010D00001C18FF102C190F103C191F11A0EA4EC8C
:1010E00007F0E8CF00F11B0EA4EC07F0E8CF01F108
:1010F0001C0EA4EC07F0E8CF02F11D0EA4EC07F0E3
:10110000E8CF03F1010103AFB4EF08F07CEC1FF06E
:101110001A0E0C6E00C10BF08DEC07F01B0E0C6E5E
:1011200001C10BF08DEC07F01C0E0C6E02C10BF030
:101130008DEC07F01D0E0C6E03C10BF08DEC07F06B
:101140001A0EA4EC07F0E8CF00F11B0EA4EC07F098
:10115000E8CF01F11C0EA4EC07F0E8CF02F11D0E60
:10116000A4EC07F0E8CF03F100C192F101C193F1C3
:1011700002C194F103C195F1240EAC6E900EAB6EDA
:10118000240EAC6E080EB86E000EB06E1F0EAF6E61
:101190000401806B816B0F01900EAB6E0F019D8A75
:1011A0000301806B816BC26B8B92C0EC24F0C0ECAE
:1011B00024F01CEC26F0A1EC22F0200EA4EC07F0A9
:1011C000E8CF2FF505012F51FF0AD8A4EFEF08F063
:1011D0002F6B200E0C6E2FC50BF08DEC07F0050168
:1011E000010E306F3C0E316F250EA4EC07F0E8CFF6
:1011F00000F1260EA4EC07F0E8CF01F1270EA4ECD5
:1012000007F0E8CF02F1280EA4EC07F0E8CF03F1D5
:10121000010103AF26EF09F07CEC1FF0250E0C6EE8
:1012200000C10BF08DEC07F0260E0C6E01C10BF027
:101230008DEC07F0270E0C6E02C10BF08DEC07F061
:10124000280E0C6E03C10BF08DEC07F000C153F5B6
:1012500001C154F502C155F503C156F500C157F55A
:1012600001C158F502C159F503C15AF5290EA4EC84
:1012700007F0E8CF5BF505015C515B5DD8A05BC56D
:101280005CF505012F51020A0EE181B853EF09F018
:1012900005015C2F50EF09F05BC55CF553EF09F0D9
:1012A00081BA5BEF26F0210EA4EC07F0E8CF00F145
:1012B000220EA4EC07F0E8CF01F1230EA4EC07F016
:1012C000E8CF02F1240EA4EC07F0E8CF03F101010E
:1012D00003AF99EF09F07CEC1FF0210E0C6E00C1FA
:1012E0000BF08DEC07F0220E0C6E01C10BF08DECB3
:1012F00007F0230E0C6E02C10BF08DEC07F0240EEC
:101300000C6E03C10BF08DEC07F0210EA4EC07F07E
:10131000E8CF00F1220EA4EC07F0E8CF01F1230E94
:10132000A4EC07F0E8CF02F1240EA4EC07F0E8CF1C
:1013300003F100C15DF501C15EF502C15FF503C1B6
:1013400060F5D8EC21F09AEC20F0EAEC1FF00501F2
:101350002F51030A12E005012F51040A1DE0050177
:101360002F51050A24E005012F51060A32E005013C
:101370002F51070A38E0FCEF09F0ACC500F101017C
:101380000F0E001701010051000A36E00101005163
:10139000050A32E0F9EF09F0ACC500F101010F0ECA
:1013A000001701010051000A27E0F9EF09F00501DB
:1013B000AC51000A21E00501AC51150A1DE0050100
:1013C000AC51300A19E00501AC51450A15E0F9EFBE
:1013D00009F00501AC51000A0FE00501AC51300ADB
:1013E0000BE0F9EF09F00501AC51000A05E0F9EF57
:1013F00009F081BA5BEF26F007900001F28EF28CC3
:1014000007B0CAEF1BF00FB0ABEF16F00FB86FEFDD
:1014100010F00301805181197F0BD8B4CAEF1BF083
:1014200013EE00F081517F0BE126812BE7CFE8FF1F
:10143000E00BD8B4CAEF1BF023EE82F0C2513F0B91
:10144000D926E7CFDFFFC22BDF50780AD8A4CAEF36
:101450001BF007808EC100F18FC101F190C102F134
:1014600091C103F10101040E046F000E056F000E1F
:10147000066F000E076F81EC1EF000AF49EF0AF017
:101480000101030E8E6F000E8F6F000E906F000E25
:10149000916F03018251720AD8B4ABEF16F08251FA
:1014A000520AD8B4ABEF16F08251750AD8B4ABEF3C
:1014B00016F08251630AD8B486EF18F08251690A97
:1014C000D8B466EF13F082517A0AD8B479EF14F0E9
:1014D0008251490AD8B405EF13F08251500AD8B4AA
:1014E00023EF12F08251700AD8B466EF12F08251E5
:1014F000540AD8B491EF12F08251740AD8B4D7EFDD
:1015000012F08251730AD8B4DBEF15F08251530AFE
:10151000D8B440EF16F082514C0AD8B4A6EF0AF0C6
:10152000BBEF18F0040114EE00F080517F0BE126B0
:1015300082C4E7FF802B120004010D0E826F92EC33
:101540000AF00A0E826F92EC0AF012000301835136
:10155000300AD8B467EF0DF003018351310AD8B4D3
:1015600075EF0EF003018351320AD8B4E3EF0EF0A9
:1015700003018351330AD8B4F3EF0EF00301835112
:10158000340AD8B403EF0FF003018351350AD8B4FD
:1015900074EF10F003018351360AD8B4A2EF10F0B3
:1015A00003018351460AD8B4C8EF0FF003018351F9
:1015B0004D0AD8B4E0EF0BF0030183516D0AD8B4A3
:1015C000FAEF0BF0030183515A0AD8B4EFEF0DF094
:1015D00003018351490AD8B4A2EF11F003018351EA
:1015E000500AD8B4D4EF10F003018351540AD8B490
:1015F0004DEF11F003018351630AD8B41AEF0CF0D8
:1016000003018351430AD8B412EF0DF00301835153
:10161000730AD8B418EF0CF003018351610AD8B4EF
:101620002DEF0BF003018351650AD8B4B7EF0DF02D
:1016300003018351450AD8B4C5EF0DF0030183516E
:10164000620AD8B4D3EF0DF003018351420AD8B433
:10165000E1EF0DF0D8A4BBEF18F004014C0E826F3F
:1016600092EC0AF00401610E826F92EC0AF09AEC9F
:1016700020F004012C0E826F92EC0AF07CEC1FF03B
:10168000ABC500F101011FEC1FF031C182F4040170
:10169000300E822792EC0AF032C182F40401300E3F
:1016A000822792EC0AF033C182F40401300E8227C3
:1016B00092EC0AF004012C0E826F92EC0AF07CECA2
:1016C0001FF0ACC500F101011FEC1FF031C182F425
:1016D0000401300E822792EC0AF032C182F4040138
:1016E000300E822792EC0AF033C182F40401300EEE
:1016F000822792EC0AF004012C0E826F92EC0AF021
:101700007CEC1FF0ADC500F101011FEC1FF031C1F1
:1017100082F40401300E822792EC0AF032C182F486
:101720000401300E822792EC0AF033C182F40401E6
:10173000300E822792EC0AF004012C0E826F92EC9C
:101740000AF07CEC1FF0AEC500F101011FEC1FF0A8
:1017500031C182F40401300E822792EC0AF032C1CA
:1017600082F40401300E822792EC0AF033C182F435
:101770000401300E822792EC0AF004012C0E826FD5
:1017800092EC0AF07CEC1FF0B3C500F101011FECF4
:101790001FF031C182F40401300E822792EC0AF06E
:1017A00032C182F40401300E822792EC0AF033C178
:1017B00082F40401300E822792EC0AF0D0EF10F090
:1017C000BDEC1FF084C333F1CAEC1FF041EC1FF0F5
:1017D000200E0C6E00C10BF08DEC07F000C12FF550
:1017E00005012F51000A06E005012F51010A02E010
:1017F00040EC21F004014C0E826F92EC0AF00401DF
:101800004D0E826F92EC0AF004012C0E826F92EC66
:101810000AF07CEC1FF02FC500F11FEC1FF033C164
:1018200082F40401300E822792EC0AF0D0EF10F01F
:101830005BEF26F004014C0E826F92EC0AF004017B
:10184000630E826F92EC0AF0EAEC1FF004012C0E9A
:10185000826F92EC0AF02FEC0CF0D0EF10F07CECE1
:101860001FF0B1C500F10101003B0F0E00171FEC86
:101870001FF033C182F40401300E822792EC0AF08B
:10188000B1C500F101010F0E010100171FEC1FF09F
:1018900033C182F40401300E822792EC0AF0040175
:1018A0002D0E826F92EC0AF0B0C500F10101003BF1
:1018B0000F0E00171FEC1FF033C182F40401300E2D
:1018C000822792EC0AF0B0C500F101010F0E010170
:1018D00000171FEC1FF033C182F40401300E822781
:1018E00092EC0AF004012D0E826F92EC0AF0AFC563
:1018F00000F10101003B0F0E00171FEC1FF033C178
:1019000082F40401300E822792EC0AF0AFC500F198
:1019100001010F0E010100171FEC1FF033C182F40B
:101920000401300E822792EC0AF00401200E826F2F
:1019300092EC0AF0AEC500F10F0E010100171FEC8A
:101940001FF033C182F40401300E822792EC0AF0BA
:101950000401200E826F92EC0AF0ADC500F1010186
:101960000101003B0F0E00171FEC1FF033C182F482
:101970000401300E822792EC0AF0ADC500F101019E
:101980000F0E010100171FEC1FF033C182F4040198
:10199000300E822792EC0AF004013A0E826F92EC2C
:1019A0000AF0ACC500F10101003B0F0E00171FEC5F
:1019B0001FF033C182F40401300E822792EC0AF04A
:1019C000ACC500F101010F0E010100171FEC1FF063
:1019D00033C182F40401300E822792EC0AF0040134
:1019E0003A0E826F92EC0AF0ABC500F10101003BA8
:1019F0000F0E00171FEC1FF033C182F40401300EEC
:101A0000822792EC0AF0ABC500F101010F0E00171E
:101A10001FEC1FF033C182F40401300E822792ECD8
:101A20000AF0120084C3E8FF0F0BE83AE8CFB1F5E3
:101A300085C3E8FF0F0B0501B11387C3E8FF0F0B48
:101A4000E83AE8CFB0F588C3E8FF0F0B0501B01303
:101A50008AC3E8FF0F0BE83AE8CFAFF58BC3E8FF86
:101A60000F0B0501AF138DC3E8FF0F0BE8CFAEF5E9
:101A70008FC3E8FF0F0BE83AE8CFADF590C3E8FF5E
:101A80000F0B0501AD1392C3E8FF0F0BE83AE8CF47
:101A9000ACF593C3E8FF0F0B0501AC1395C3E8FF4A
:101AA0000F0BE83AE8CFABF596C3E8FF0F0B050143
:101AB000AB1349EC20F004014C0E826F92EC0AF05B
:101AC0000401430E826F92EC0AF024EF0CF00784BD
:101AD0001CEC26F07CEC1FF02DC500F11FEC1FF074
:101AE00004014C0E826F92EC0AF00401300E826FFA
:101AF00092EC0AF004012C0E826F92EC0AF031C1D4
:101B000082F40401300E822792EC0AF032C182F492
:101B10000401300E822792EC0AF033C182F40401F2
:101B2000300E822792EC0AF004012C0E826F92ECA8
:101B30000AF07CEC1FF02EC500F11FEC1FF031C144
:101B400082F40401300E822792EC0AF032C182F452
:101B50000401300E822792EC0AF033C182F40401B2
:101B6000300E822792EC0AF00794D0EF10F00401B7
:101B70004C0E826F92EC0AF00401650E826F92ECBB
:101B80000AF029EC22F0D0EF10F004014C0E826F25
:101B900092EC0AF00401450E826F92EC0AF046ECDA
:101BA00022F0D0EF10F004014C0E826F92EC0AF09C
:101BB0000401620E826F92EC0AF080EC22F0D0EF0A
:101BC00010F004014C0E826F92EC0AF00401420EF8
:101BD000826F92EC0AF063EC22F0D0EF10F0040177
:101BE0004C0E826F92EC0AF004015A0E826F92EC56
:101BF0000AF004012C0E826F92EC0AF01CEC26F025
:101C00007CEC1FF005012E51130A06E005012E5150
:101C1000170A0DE020EF0EF00101000E006F000E1C
:101C2000016F100E026F000E036F20EF0EF0010126
:101C3000000E006F000E016F000E026F010E036FA9
:101C40000101100E046F000E056F000E066F000EEE
:101C5000076FB2EC1EF01FEC1FF02AC182F40401E2
:101C6000300E822792EC0AF02BC182F40401300E70
:101C7000822792EC0AF02CC182F40401300E8227F4
:101C800092EC0AF02DC182F40401300E822792EC0E
:101C90000AF02EC182F40401300E822792EC0AF081
:101CA0002FC182F40401300E822792EC0AF030C179
:101CB00082F40401300E822792EC0AF031C182F4E2
:101CC0000401300E822792EC0AF032C182F4040142
:101CD000300E822792EC0AF033C182F40401300EF8
:101CE000822792EC0AF0D0EF10F0078404014C0E2A
:101CF000826F92EC0AF00401310E826F92EC0AF0CE
:101D000004012C0E826F92EC0AF025C500F126C565
:101D100001F127C502F128C503F10101100E046F7E
:101D2000000E056F000E066F000E076FB2EC1EF07E
:101D30001FEC1FF02AC182F40401300E822792ECBE
:101D40000AF02BC182F40401300E822792EC0AF0D3
:101D50002CC182F40401300E822792EC0AF02DC1CE
:101D600082F40401300E822792EC0AF02EC182F434
:101D70000401300E822792EC0AF02FC182F4040194
:101D8000300E822792EC0AF030C182F40401300E4A
:101D9000822792EC0AF031C182F40401300E8227CE
:101DA00092EC0AF032C182F40401300E822792ECE8
:101DB0000AF033C182F40401300E822792EC0AF05B
:101DC0000794D0EF10F0078404014C0E826F92EC60
:101DD0000AF00401320E826F92EC0AF076EC24F0E5
:101DE0000794D0EF10F0078404014C0E826F92EC40
:101DF0000AF00401330E826F92EC0AF0D3EC24F067
:101E0000079480EF0EF0078404014C0E826F92EC71
:101E10000AF00401340E826F92EC0AF004012C0ED9
:101E2000826F92EC0AF0BDEC1FF084C32AF185C3E7
:101E30002BF186C32CF187C32DF188C32EF189C302
:101E40002FF18AC330F18BC331F18CC332F18DC3D2
:101E500033F10101296BCAEC1FF041EC1FF0100EA9
:101E6000046F000E056F000E066F000E076F92ECF8
:101E70001EF000C121F501C122F502C123F503C105
:101E800024F5CFEC25F034C5ABF535C5ACF536C53A
:101E9000ADF537C5AEF538C5AFF539C5B0F53AC5BE
:101EA000B1F52FEC0CF004012C0E826F92EC0AF0CD
:101EB0003BC500F13CC501F13DC502F13EC503F152
:101EC0000101000E046F000E056F010E066F000E7B
:101ED000076FB2EC1EF01FEC1FF0296772EF0FF0D6
:101EE00077EF0FF004012D0E826F92EC0AF030C1F3
:101EF00082F40401300E822792EC0AF031C182F4A0
:101F00000401300E822792EC0AF004012E0E826F3B
:101F100092EC0AF032C182F40401300E822792EC76
:101F20000AF033C182F40401300E822792EC0AF0E9
:101F300004012C0E826F92EC0AF07CEC1FF03FC57E
:101F400000F140C501F1E5EC19F004012C0E826F9F
:101F500092EC0AF07CEC1FF041C500F11FEC1FF081
:101F600031C182F40401300E822792EC0AF032C1B2
:101F700082F40401300E822792EC0AF033C182F41D
:101F80000401300E822792EC0AF00794D0EF10F093
:101F9000BDEC1FF085C32AF186C32BF187C32CF15A
:101FA00088C32DF189C32EF18AC32FF18BC330F181
:101FB0008CC331F18DC332F18EC333F10101296B32
:101FC000CAEC1FF041EC1FF00101010E046F000E7E
:101FD000056F000E066F000E076F81EC1EF0100EED
:101FE000046F000E056F000E066F000E076F92EC77
:101FF0001EF000C129F501C12AF502C12BF503C16C
:102000002CF5FFEC23F004014C0E826F92EC0AF0E9
:102010000401460E826F92EC0AF004012C0E826FCE
:1020200092EC0AF025C500F126C501F127C502F1A1
:1020300028C503F10101100E046F000E056F000E9C
:10204000066F000E076FB2EC1EF01FEC1FF02AC1E6
:1020500082F40401300E822792EC0AF02BC182F444
:102060000401300E822792EC0AF02CC182F40401A4
:10207000300E822792EC0AF02DC182F40401300E5A
:10208000822792EC0AF02EC182F40401300E8227DE
:1020900092EC0AF02FC182F40401300E822792ECF8
:1020A0000AF030C182F40401300E822792EC0AF06B
:1020B00031C182F40401300E822792EC0AF032C161
:1020C00082F40401300E822792EC0AF033C182F4CC
:1020D0000401300E822792EC0AF0D0EF10F00F9836
:1020E000D3EC24F0BBEF18F004014C0E826F92EC9D
:1020F0000AF00401350E826F92EC0AF004012C0EF6
:10210000826F92EC0AF07CEC1FF00784B5C500F1F9
:1021100007941FEC1FF031C182F40401300E8227B6
:1021200092EC0AF032C182F40401300E822792EC64
:102130000AF033C182F40401300E822792EC0AF0D7
:10214000D0EF10F096EC24F07CEC1FF033C500F1DA
:102150001FEC1FF004014C0E826F92EC0AF0040198
:10216000360E826F92EC0AF004012C0E826F92EC14
:102170000AF031C182F40401300E822792EC0AF099
:1021800032C182F40401300E822792EC0AF033C18E
:1021900082F40401300E822792EC0AF0D0EF10F0A6
:1021A0009CEC0AF0BBEF18F004014C0E826F92EC2D
:1021B0000AF00401500E826F92EC0AF004012C0E1A
:1021C000826F92EC0AF085C32AF186C32BF187C394
:1021D0002CF188C32DF189C32EF18AC32FF18BC353
:1021E00030F18CC331F18DC332F18EC333F1010173
:1021F000CAEC1FF041EC1FF003018451530A0DE0BB
:10220000030184514D0A38E00401780E826F92EC8C
:102210000AF09CEC0AF0BBEF18F00401530E826F39
:1022200092EC0AF0250E0C6E00C10BF08DEC07F05D
:10223000260E0C6E01C10BF08DEC07F0270E0C6E14
:1022400002C10BF08DEC07F0280E0C6E03C10BF0F1
:102250008DEC07F000C153F501C154F502C155F5ED
:1022600003C156F500C157F501C158F502C159F532
:1022700003C15AF5B1EF11F004014D0E826F92ECDB
:102280000AF0290E0C6E00C10BF08DEC07F000C1B6
:102290005BF500C15CF5B1EF11F004014C0E826FEB
:1022A00092EC0AF00401540E826F92EC0AF00401E1
:1022B0002C0E826F92EC0AF084C32AF185C32BF1B5
:1022C00086C32CF187C32DF188C32EF189C32FF16A
:1022D0008AC330F18BC331F18DC332F18EC333F138
:1022E0000101CAEC1FF041EC1FF00101000E046F68
:1022F000000E056F010E066F000E076F92EC1EF0C8
:10230000210E0C6E00C10BF08DEC07F0220E0C6E4E
:1023100001C10BF08DEC07F0230E0C6E02C10BF027
:102320008DEC07F0240E0C6E03C10BF08DEC07F062
:1023300000C15DF501C15EF502C15FF503C160F545
:10234000B1EF11F004014C0E826F92EC0AF004011F
:10235000490E826F92EC0AF004012C0E826F92EC0F
:102360000AF0250EA4EC07F0E8CF00F1260EA4EC4D
:1023700007F0E8CF01F1270EA4EC07F0E8CF02F157
:10238000280EA4EC07F0E8CF03F11FEC1FF002ECDD
:102390001DF00401730E826F92EC0AF004012C0E02
:1023A000826F92EC0AF07CEC1FF0290EA4EC07F08F
:1023B000E8CF00F11FEC1FF002EC1DF00401730EDA
:1023C000826F92EC0AF004012C0E826F92EC0AF0FC
:1023D00057C500F158C501F159C502F15AC503F1BD
:1023E0001FEC1FF002EC1DF00401730E826F92ECE3
:1023F0000AF004012C0E826F92EC0AF07CEC1FF0C4
:102400005CC500F11FEC1FF002EC1DF004016D0E25
:10241000826F92EC0AF004012C0E826F92EC0AF0AB
:102420005DC500F15EC501F15FC502F160C503F154
:10243000D6EC18F004012C0E826F92EC0AF09CECA2
:102440000AF0BBEF18F083C32AF184C32BF185C3D4
:102450002CF186C32DF187C32EF188C32FF189C3D8
:1024600030F18AC331F18BC332F18CC333F10101F6
:10247000CAEC1FF041EC1FF0160E0C6E00C10BF001
:102480008DEC07F0170E0C6E01C10BF08DEC07F010
:10249000180E0C6E02C10BF08DEC07F0190E0C6ECD
:1024A00003C10BF08DEC07F000C18AF101C18BF183
:1024B00002C18CF103C18DF100C18EF101C18FF118
:1024C00002C190F103C191F105EF13F083C32AF12A
:1024D00084C32BF185C32CF186C32DF187C32EF164
:1024E00088C32FF189C330F18AC331F18BC332F134
:1024F0008CC333F10101CAEC1FF041EC1FF000C1A5
:102500008AF101C18BF102C18CF103C18DF100C1CF
:102510008EF101C18FF102C190F103C191F105EF7C
:1025200013F083C32AF184C32BF185C32CF186C336
:102530002DF187C32EF188C32FF189C330F18AC3EF
:1025400031F18CC332F18DC333F10101CAEC1FF0BC
:1025500041EC1FF00101000E046F000E056F010E2B
:10256000066F000E076F92EC1EF01A0E0C6E00C183
:102570000BF08DEC07F01B0E0C6E01C10BF08DEC17
:1025800007F01C0E0C6E02C10BF08DEC07F01D0E57
:102590000C6E03C10BF08DEC07F000C192F101C18C
:1025A00093F102C194F103C195F105EF13F083C3D8
:1025B0002AF184C32BF185C32CF186C32DF187C387
:1025C0002EF188C32FF189C330F18AC331F18CC356
:1025D00032F18DC333F10101CAEC1FF041EC1FF061
:1025E0000101000E046F000E056F010E066F000E54
:1025F000076F92EC1EF000C192F101C193F102C18C
:1026000094F103C195F105EF13F0160EA4EC07F059
:10261000E8CF00F1170EA4EC07F0E8CF01F1180E97
:10262000A4EC07F0E8CF02F1190EA4EC07F0E8CF14
:1026300003F11FEC1FF002EC1DF00401730E826F1A
:1026400092EC0AF004012C0E826F92EC0AF08AC11F
:1026500000F18BC101F18CC102F18DC103F11FECBE
:102660001FF002EC1DF00401730E826F92EC0AF071
:1026700004012C0E826F92EC0AF01A0EA4EC07F003
:10268000E8CF00F11B0EA4EC07F0E8CF01F11C0E1F
:10269000A4EC07F0E8CF02F11D0EA4EC07F0E8CFA0
:1026A00003F1D6EC18F004012C0E826F92EC0AF0C4
:1026B00092C100F193C101F194C102F195C103F1FE
:1026C000D6EC18F09CEC0AF0BBEF18F00401690E90
:1026D000826F92EC0AF004012C0E826F92EC0AF0E9
:1026E0000101040E006F000E016F000E026F000E5C
:1026F000036F1FEC1FF02CC182F40401300E8227FF
:1027000092EC0AF02DC182F40401300E822792EC83
:102710000AF02EC182F40401300E822792EC0AF0F6
:102720002FC182F40401300E822792EC0AF030C1EE
:1027300082F40401300E822792EC0AF031C182F457
:102740000401300E822792EC0AF032C182F40401B7
:10275000300E822792EC0AF033C182F40401300E6D
:10276000822792EC0AF004012C0E826F92EC0AF0A0
:102770000101060E006F000E016F000E026F000EC9
:10278000036F1FEC1FF02CC182F40401300E82276E
:1027900092EC0AF02DC182F40401300E822792ECF3
:1027A0000AF02EC182F40401300E822792EC0AF066
:1027B0002FC182F40401300E822792EC0AF030C15E
:1027C00082F40401300E822792EC0AF031C182F4C7
:1027D0000401300E822792EC0AF032C182F4040127
:1027E000300E822792EC0AF033C182F40401300EDD
:1027F000822792EC0AF004012C0E826F92EC0AF010
:102800000101210E006F000E016F000E026F000E1D
:10281000036F1FEC1FF02CC182F40401300E8227DD
:1028200092EC0AF02DC182F40401300E822792EC62
:102830000AF02EC182F40401300E822792EC0AF0D5
:102840002FC182F40401300E822792EC0AF030C1CD
:1028500082F40401300E822792EC0AF031C182F436
:102860000401300E822792EC0AF032C182F4040196
:10287000300E822792EC0AF033C182F40401300E4C
:10288000822792EC0AF004012C0E826F92EC0AF07F
:10289000200EF86EF76AF66A04010900F5CF82F49B
:1028A00092EC0AF00900F5CF82F492EC0AF00900EC
:1028B000F5CF82F492EC0AF00900F5CF82F492ECA5
:1028C0000AF00900F5CF82F492EC0AF00900F5CF86
:1028D00082F492EC0AF00900F5CF82F492EC0AF04F
:1028E0000900F5CF82F492EC0AF09CEC0AF0BBEF01
:1028F00018F08351630AD8A4BBEF18F08451610A21
:10290000D8A4BBEF18F085516C0AD8A4BBEF18F01F
:102910008651410A42E08651440A1BE08651420A30
:10292000D8B4E0EF14F08651350AD8B445EF1AF068
:102930008651360AD8B49AEF1AF08651370AD8B4BD
:1029400003EF1BF08651380AD8B461EF1BF0BBEFE0
:1029500018F00798079A04017A0E826F92EC0AF039
:102960000401780E826F92EC0AF00401640E826F0B
:1029700092EC0AF081A8C4EF14F00401550E826FA6
:1029800092EC0AF0C9EF14F004014C0E826F92EC45
:102990000AF09CEC0AF0BBEF18F00788079A0401D4
:1029A0007A0E826F92EC0AF00401410E826F92EC73
:1029B0000AF00401610E826F92EC0AF0BAEF14F093
:1029C0000798078A04017A0E826F92EC0AF00401DC
:1029D000420E826F92EC0AF00401610E826F92EC5B
:1029E0000AF0BAEF14F001016667FEEF14F06767B2
:1029F000FEEF14F06867FEEF14F0696716EF15F04C
:102A00004F670AEF15F050670AEF15F051670AEFAC
:102A100015F0526716EF15F00101000E006F000E61
:102A2000016F000E026F000E036F12000101620EB3
:102A3000046F010E056F000E066F000E076F66C172
:102A400000F167C101F168C102F169C103F181ECD4
:102A50001EF003BF9AEF15F00101000E046FA80EDF
:102A6000056F550E066F020E076F66C100F167C154
:102A700001F168C102F169C103F166C186F167C164
:102A800087F168C188F169C189F181EC1EF003BF4B
:102A900053EF15F00101000E866FA80E876F550EDB
:102AA000886F020E896F0E0EA4EC07F0E8CF18F1C4
:102AB0000F0EA4EC07F0E8CF19F1100EA4EC07F00C
:102AC000E8CF1AF1110EA4EC07F0E8CF1BF1CAEC25
:102AD0001DF086C104F187C105F188C106F189C1E5
:102AE00007F181EC1EF007828EEC1DF0CAEC1DF0A0
:102AF00007928EEC1DF086C100F187C101F188C1FB
:102B000002F189C103F107928EEC1DF0CC0E046F27
:102B1000E00E056F870E066F050E076F81EC1EF045
:102B200000C118F101C119F102C11AF103C11BF171
:102B3000D2EF15F00101800E006F1A0E016F060E24
:102B4000026F000E036F4FC104F150C105F151C176
:102B500006F152C107F181EC1EF003AFB3EF15F09F
:102B60007CEC1FF012000E0EA4EC07F0E8CF18F179
:102B70000F0EA4EC07F0E8CF19F1100EA4EC07F04B
:102B8000E8CF1AF1110EA4EC07F0E8CF1BF14FC10A
:102B900000F150C101F151C102F152C103F10782AC
:102BA0008EEC1DF018C100F119C101F11AC102F13A
:102BB0001BC103F112000401730E826F92EC0AF044
:102BC00004012C0E826F92EC0AF0078462C166F158
:102BD00063C167F164C168F165C169F14BC14FF12F
:102BE0004CC150F14DC151F14EC152F157C159F193
:102BF00058C15AF1079401EC16F09CEC0AF0BBEFB7
:102C000018F066C100F167C101F168C102F169C144
:102C100003F101011FEC1FF002EC1DF00401630E33
:102C2000826F92EC0AF004012C0E826F92EC0AF093
:102C30004FC100F150C101F151C102F152C103F184
:102C400001011FEC1FF002EC1DF00401660E826F03
:102C500092EC0AF004012C0E826F92EC0AF07CECEC
:102C60001FF059C100F15AC101F101011FEC1FF021
:102C700002EC1DF00401740E826F92EC0AF0120057
:102C800010820401530E826F92EC0AF004012C0EA4
:102C9000826F92EC0AF083C32AF184C32BF185C3BF
:102CA0002CF186C32DF187C32EF188C32FF189C380
:102CB00030F18AC331F18BC332F18CC333F101019E
:102CC000CAEC1FF041EC1FF000C166F101C167F1D1
:102CD00002C168F103C169F18EC32AF18FC32BF1E0
:102CE00090C32CF191C32DF192C32EF193C32FF118
:102CF00094C330F195C331F196C332F197C333F1E8
:102D00000101CAEC1FF041EC1FF000C14FF101C1FD
:102D100050F102C151F103C152F1BDEC1FF099C352
:102D20002FF19AC330F19BC331F19CC332F19DC3A3
:102D300033F10101CAEC1FF041EC1FF000C159F161
:102D400001C15AF101EC16F004012C0E826F92ECD5
:102D50000AF0B2EF16F08251520A03E10F82B2EF8D
:102D600016F00F928251750A03E11084B9EF16F044
:102D700010948251550A03E11086C0EF16F01096A8
:102D8000078410B21DEF17F010A409EF17F0B6C1B9
:102D900066F1B7C167F1B8C168F1B9C169F1BAC1EB
:102DA0006AF1BBC16BF1BCC16CF1BDC16DF1BEC1BB
:102DB0006EF1BFC16FF1C0C170F1C1C171F1C2C18B
:102DC00072F1C3C173F1C4C174F1C5C175F1C6C15B
:102DD00076F1C7C177F1C8C178F1C9C179F1CAC12B
:102DE0007AF1CBC17BF1CCC17CF1CDC17DF1CEC1FB
:102DF0007EF1CFC17FF1D0C180F1D1C181F1D2C1CB
:102E000082F1D3C183F1D4C184F1D5C185F111EF31
:102E100017F062C166F163C167F164C168F165C111
:102E200069F14BC14FF14CC150F14DC151F14EC14F
:102E300052F157C159F158C15AF107940FA03FEF11
:102E400017F0010192672CEF17F093672CEF17F042
:102E500094672CEF17F0956730EF17F03FEF17F0FE
:102E6000F3EC14F092C104F193C105F194C106F1A1
:102E700095C107F181EC1EF003BF83EF18F0F3EC6E
:102E800014F00101000E046F000E056F010E066FB5
:102E9000000E076FB2EC1EF010A456EF17F00401FD
:102EA000750E826F92EC0AF05BEF17F00401720E60
:102EB000826F92EC0AF004012C0E826F92EC0AF001
:102EC0001FEC1FF029676AEF17F00401200E826FD4
:102ED0006DEF17F004012D0E826F92EC0AF030C1F5
:102EE00082F40401300E822792EC0AF031C182F4A0
:102EF0000401300E822792EC0AF004012E0E826F3C
:102F000092EC0AF032C182F40401300E822792EC76
:102F10000AF033C182F40401300E822792EC0AF0E9
:102F200004016D0E826F92EC0AF004012C0E826F88
:102F300092EC0AF04FC100F150C101F151C102F110
:102F400052C103F101011FEC1FF002EC1DF004015E
:102F5000480E826F92EC0AF004017A0E826F92ECB6
:102F60000AF004012C0E826F92EC0AF066C100F1A7
:102F700067C101F168C102F169C103F101011FECF0
:102F80001FF002EC1DF00401630E826F92EC0AF058
:102F900004012C0E826F92EC0AF066C100F167C149
:102FA00001F168C102F169C103F101010A0E046F68
:102FB000000E056F000E066F000E076F92EC1EF0FC
:102FC000000E046F120E056F000E066F000E076FE5
:102FD000B2EC1EF01FEC1FF02AC182F40401300E87
:102FE000822792EC0AF02BC182F40401300E822772
:102FF00092EC0AF02CC182F40401300E822792EC8C
:103000000AF02DC182F40401300E822792EC0AF0FE
:103010002EC182F40401300E822792EC0AF02FC1F7
:1030200082F40401300E822792EC0AF030C182F45F
:103030000401300E822792EC0AF004012E0E826FFA
:1030400092EC0AF031C182F40401300E822792EC36
:103050000AF032C182F40401300E822792EC0AF0A9
:1030600033C182F40401300E822792EC0AF004018D
:10307000730E826F92EC0AF004012C0E826F92ECB8
:103080000AF07CEC1FF059C100F15AC101F1E5ECE6
:1030900019F00FB24FEF18F00FA081EF18F00401F4
:1030A0002C0E826F92EC0AF0200EF86EF76AF66A28
:1030B00004010900F5CF82F492EC0AF00900F5CF83
:1030C00082F492EC0AF00900F5CF82F492EC0AF057
:1030D0000900F5CF82F492EC0AF00900F5CF82F4F2
:1030E00092EC0AF00900F5CF82F492EC0AF00900A4
:1030F000F5CF82F492EC0AF00900F5CF82F492EC5D
:103100000AF09CEC0AF00F90BBEF18F00401630E7C
:10311000826F92EC0AF004012C0E826F92EC0AF09E
:10312000C1EC18F004012C0E826F92EC0AF034EC22
:1031300019F004012C0E826F92EC0AF0B0EC19F039
:1031400004012C0E826F92EC0AF00101F80E006F60
:10315000CD0E016F660E026F030E036FD6EC18F0F2
:1031600004012C0E826F92EC0AF0C6EC19F09CEC74
:103170000AF0BBEF18F00301C26B07901092CAEF80
:103180001BF0D8900E0EA4EC07F0E8CF00F10F0E64
:10319000A4EC07F0E8CF01F1100EA4EC07F0E8CFA3
:1031A00002F1110EA4EC07F0E8CF03F10101000ECB
:1031B000046F000E056F010E066F000E076FB2EC74
:1031C0001EF01FEC1FF02AC182F40401300E82278A
:1031D00092EC0AF02BC182F40401300E822792ECAB
:1031E0000AF02CC182F40401300E822792EC0AF01E
:1031F0002DC182F40401300E822792EC0AF02EC118
:1032000082F40401300E822792EC0AF02FC182F47E
:103210000401300E822792EC0AF030C182F40401DE
:10322000300E822792EC0AF031C182F40401300E94
:10323000822792EC0AF004012E0E826F92EC0AF0C3
:1032400032C182F40401300E822792EC0AF033C1BD
:1032500082F40401300E822792EC0AF004016D0E14
:10326000826F92EC0AF01200120EA4EC07F0E8CF85
:1032700000F1130EA4EC07F0E8CF01F1140EA4EC5A
:1032800007F0E8CF02F1150EA4EC07F0E8CF03F148
:1032900001010A0E046F000E056F000E066F000E8E
:1032A000076F92EC1EF0000E046F120E056F000EF9
:1032B000066F000E076FB2EC1EF01FEC1FF02AC164
:1032C00082F40401300E822792EC0AF02BC182F4C2
:1032D0000401300E822792EC0AF02CC182F4040122
:1032E000300E822792EC0AF02DC182F40401300ED8
:1032F000822792EC0AF02EC182F40401300E82275C
:1033000092EC0AF02FC182F40401300E822792EC75
:103310000AF030C182F40401300E822792EC0AF0E8
:1033200004012E0E826F92EC0AF031C182F4040186
:10333000300E822792EC0AF032C182F40401300E82
:10334000822792EC0AF033C182F40401300E822706
:1033500092EC0AF00401730E826F92EC0AF01200F4
:103360000A0EA4EC07F0E8CF00F10B0EA4EC07F076
:10337000E8CF01F10C0EA4EC07F0E8CF02F10D0E3E
:10338000A4EC07F0E8CF03F1E5EF19F0060EA4EC8A
:1033900007F0E8CF00F1070EA4EC07F0E8CF01F149
:1033A000080EA4EC07F0E8CF02F1090EA4EC07F038
:1033B000E8CF03F1E5EF19F001017CEC1FF0078481
:1033C00057C100F158C101F107940101E80E046FE3
:1033D000800E056F000E066F000E076F92EC1EF058
:1033E000000E046F040E056F000E066F000E076FCF
:1033F000B2EC1EF0880E046F130E056F000E066F00
:10340000000E076F81EC1EF00A0E046F000E056FB0
:10341000000E066F000E076FB2EC1EF01FEC1FF0DF
:103420000101296719EF1AF00401200E826F1CEFC9
:103430001AF004012D0E826F92EC0AF030C182F472
:103440000401300E822792EC0AF031C182F40401AB
:10345000300E822792EC0AF032C182F40401300E61
:10346000822792EC0AF004012E0E826F92EC0AF091
:1034700033C182F40401300E822792EC0AF0040179
:10348000430E826F92EC0AF0120087C32AF188C3C0
:103490002BF189C32CF18AC32DF18BC32EF18CC380
:1034A0002FF18DC330F18EC331F190C332F191C34E
:1034B00033F10101296BCAEC1FF041EC1FF001014F
:1034C000000E046F000E056F010E066F000E076FF1
:1034D00092EC1EF00E0E0C6E00C10BF08DEC07F09E
:1034E0000F0E0C6E01C10BF08DEC07F0100E0C6E80
:1034F00002C10BF08DEC07F0110E0C6E03C10BF046
:103500008DEC07F004017A0E826F92EC0AF0040150
:103510002C0E826F92EC0AF00401350E826F92EC51
:103520000AF004012C0E826F92EC0AF0C1EC18F044
:10353000C9EF14F087C32AF188C32BF189C32CF19A
:103540008AC32DF18BC32EF18CC32FF18DC330F1C3
:103550008EC331F190C332F191C333F10101296B74
:10356000CAEC1FF041EC1FF0880E046F130E056FBC
:10357000000E066F000E076F86EC1EF0000E046F43
:10358000040E056F000E066F000E076F92EC1EF022
:103590000101E80E046F800E056F000E066F000E2D
:1035A000076FB2EC1EF00A0E0C6E00C10BF08DEC32
:1035B00007F00B0E0C6E01C10BF08DEC07F00C0E3A
:1035C0000C6E02C10BF08DEC07F00D0E0C6E03C1FA
:1035D0000BF08DEC07F004017A0E826F92EC0AF08A
:1035E00004012C0E826F92EC0AF00401360E826FF9
:1035F00092EC0AF004012C0E826F92EC0AF0B0EC0F
:1036000019F0C9EF14F087C32AF188C32BF189C3DD
:103610002CF18AC32DF18BC32EF18CC32FF18DC3F6
:1036200030F18FC331F190C332F191C333F1010115
:10363000CAEC1FF041EC1FF0000E046F120E056F74
:10364000000E066F000E076F92EC1EF001010A0ECD
:10365000046F000E056F000E066F000E076FB2ECD0
:103660001EF0120E0C6E00C10BF08DEC07F0130E65
:103670000C6E01C10BF08DEC07F0140E0C6E02C144
:103680000BF08DEC07F0150E0C6E03C10BF08DECFA
:1036900007F004017A0E826F92EC0AF004012C0EFE
:1036A000826F92EC0AF00401370E826F92EC0AF0FE
:1036B00004012C0E826F92EC0AF034EC19F0C9EF81
:1036C00014F087C32AF188C32BF189C32CF18AC374
:1036D0002DF18BC32EF18CC32FF18DC330F18EC32E
:1036E00031F190C332F191C333F10101296BCAEC7E
:1036F0001FF041EC1FF0880E046F130E056F000ED3
:10370000066F000E076F86EC1EF0000E046F040EAD
:10371000056F000E066F000E076F92EC1EF00101A0
:10372000E80E046F800E056F000E066F000E076F27
:10373000B2EC1EF0060E0C6E00C10BF08DEC07F023
:10374000070E0C6E01C10BF08DEC07F0080E0C6E2D
:1037500002C10BF08DEC07F0090E0C6E03C10BF0EB
:103760008DEC07F004017A0E826F92EC0AF00401EE
:103770002C0E826F92EC0AF00401380E826F92ECEC
:103780000AF004012C0E826F92EC0AF0C6EC19F0DC
:10379000C9EF14F081A888EF1CF007A841EF1CF0D6
:1037A0000101800E006F1A0E016F060E026F000EEF
:1037B000036F4BC104F14CC105F14DC106F14EC17F
:1037C00007F181EC1EF003BF88EF1CF0FCEC1CF04D
:1037D0004BC100F14CC101F14DC102F14EC103F1E9
:1037E00007828EEC1DF018C104F119C105F11AC150
:1037F00006F11BC107F1F80E006FCD0E016F660ECA
:10380000026F030E036F81EC1EF00E0E0C6E00C1F2
:103810000BF08DEC07F00F0E0C6E01C10BF08DEC70
:1038200007F0100E0C6E02C10BF08DEC07F0110EBC
:103830000C6E03C10BF08DEC07F0078401017CECEA
:103840001FF057C100F158C101F107940A0E0C6E28
:1038500000C10BF08DEC07F00B0E0C6E01C10BF0EC
:103860008DEC07F00C0E0C6E02C10BF08DEC07F026
:103870000D0E0C6E03C10BF08DEC07F0079888EF6E
:103880001CF007AA88EF1CF0078401017CEC1FF0F4
:1038900057C100F158C101F10794060E0C6E00C12A
:1038A0000BF08DEC07F0070E0C6E01C10BF08DECE8
:1038B00007F0080E0C6E02C10BF08DEC07F0090E3C
:1038C0000C6E03C10BF08DEC07F0078462C100F1B0
:1038D00063C101F164C102F165C103F10794120EE5
:1038E0000C6E00C10BF08DEC07F0130E0C6E01C1D5
:1038F0000BF08DEC07F0140E0C6E02C10BF08DEC8A
:1039000007F0150E0C6E03C10BF08DEC07F0079A53
:103910000401805181197F0B0BE09EA809D014EEA1
:1039200000F081517F0BE126E750812B0F01AD6E36
:1039300005012F51010A13E081AAAFEF1CF0050128
:103940002F51000A0AE00FB8AFEF1CF005013067F5
:10395000AFEF1CF00FB8AFEF1CF05BEF26F081B8B3
:10396000C4EF1CF09AEC20F005012F51020A02E08E
:10397000C4EF1CF05C2FC4EF1CF05BC55CF50501C7
:10398000010E306F3C0E316F00EF0AF018C100F1EC
:1039900019C101F11AC102F11BC103F1000E046F3C
:1039A000000E056F010E066F000E076FB2EC1EF0E1
:1039B00029A1F1EF1CF02051D8B4F1EF1CF018C18F
:1039C00000F119C101F11AC102F11BC103F1000E8E
:1039D000046F000E056F0A0E066F000E076FB2EC43
:1039E0001EF012000101045100130551011306518C
:1039F00002130751031312000101186B196B1A6BA4
:103A00001B6B12002AC182F40401300E822792EC53
:103A10000AF02BC182F40401300E822792EC0AF0E6
:103A20002CC182F40401300E822792EC0AF02DC1E1
:103A300082F40401300E822792EC0AF02EC182F447
:103A40000401300E822792EC0AF02FC182F40401A7
:103A5000300E822792EC0AF030C182F40401300E5D
:103A6000822792EC0AF031C182F40401300E8227E1
:103A700092EC0AF032C182F40401300E822792ECFB
:103A80000AF033C182F40401300E822792EC0AF06E
:103A900012002FC182F40401300E822792EC0AF04A
:103AA00030C182F40401300E822792EC0AF031C159
:103AB00082F40401300E822792EC0AF032C182F4C3
:103AC0000401300E822792EC0AF033C182F4040123
:103AD000300E822792EC0AF01200060E116E060ECE
:103AE000126E060E136E112E73EF1DF0122E73EF71
:103AF0001DF0132E73EF1DF08B84020E116E020E5B
:103B0000126E020E136E112E83EF1DF0122E83EF34
:103B10001DF0132E83EF1DF08B9412000101005352
:103B200005E1015303E1025301E1002B51EC1EF0CA
:103B30007CEC1FF03951006F3A51016F420E046F57
:103B40004B0E056F000E066F000E076F92EC1EF015
:103B500000C104F101C105F102C106F103C107F181
:103B600018C100F119C101F11AC102F11BC103F121
:103B700007B2BFEF1DF086EC1EF0C1EF1DF081EC27
:103B80001EF000C118F101C119F102C11AF103C1FF
:103B90001BF112007CEC1FF059C100F15AC101F178
:103BA000060EA4EC07F0E8CF04F1070EA4EC07F032
:103BB000E8CF05F1080EA4EC07F0E8CF06F1090EF6
:103BC000A4EC07F0E8CF07F181EC1EF000C124F16E
:103BD00001C125F102C126F103C127F1290E046FAD
:103BE000000E056F000E066F000E076F92EC1EF0C0
:103BF000EE0E046F430E056F000E066F000E076F8A
:103C000086EC1EF024C104F125C105F126C106F1A0
:103C100027C107F192EC1EF000C11CF101C11DF19A
:103C200002C11EF103C11FF1120EA4EC07F0E8CF90
:103C300004F1130EA4EC07F0E8CF05F1140EA4EC88
:103C400007F0E8CF06F1150EA4EC07F0E8CF07F176
:103C50000D0E006F000E016F000E026F000E036F5D
:103C600092EC1EF0180E046F000E056F000E066F2A
:103C7000000E076FB2EC1EF01CC104F11DC105F16E
:103C80001EC106F11FC107F186EC1EF06A0E046F1B
:103C90002A0E056F000E066F000E076F81EC1EF0F6
:103CA0001200BF0EFA6E200E3A6F396BD8900037B3
:103CB000013702370337D8B062EF1EF03A2F57EFC3
:103CC0001EF039073A070353D8B412000331070B2B
:103CD00080093F6F03390F0B010F396F80EC5FF0E4
:103CE000406F390580EC5FF0405D405F396B3F33DA
:103CF000D8B0392739333FA977EF1EF04051392723
:103D000012000101A1EC1FF0D8B012000101035113
:103D10000719346F64EC1FF0D8900751031934AFC2
:103D2000800F12000101346B88EC1FF0D8A09EECCC
:103D30001FF0D8B0120073EC1FF07CEC1FF01F0EC8
:103D4000366FB4EC1FF00B35D8B064EC1FF0D8A080
:103D50000335D8B01200362FA1EF1EF034B18BEC32
:103D60001FF012000101346B0451051106110711F7
:103D70000008D8A088EC1FF0D8A09EEC1FF0D8B0A7
:103D80001200086B096B0A6B0B6BB4EC1FF01F0E73
:103D9000366FB4EC1FF007510B5DD8A4DCEF1EF0BA
:103DA00006510A5DD8A4DCEF1EF00551095DD8A4C8
:103DB000DCEF1EF00451085DD8A0EFEF1EF00451B7
:103DC000085F0551D8A0053D095F0651D8A0063D02
:103DD0000A5F0751D8A0073D0B5FD8900081362FAE
:103DE000C9EF1EF034B18BEC1FF0346B88EC1FF080
:103DF000D890B8EC1FF007510B5DD8A40CEF1FF062
:103E000006510A5DD8A40CEF1FF00551095DD8A436
:103E10000CEF1FF00451085DD8A01BEF1FF0003F0E
:103E20001BEF1FF0013F1BEF1FF0023F1BEF1FF0C6
:103E3000032BD8B4120034B18BEC1FF01200010137
:103E4000346B88EC1FF0D8B01200BDEC1FF0200ED0
:103E5000366F003701370237033711EE33F00A0EA1
:103E6000376FE7360A0EE75CD8B0E76EE552372FBA
:103E700031EF1FF0362F29EF1FF034B12981D89090
:103E8000120001010A0E346F200E366F11EE29F078
:103E90003451376F0A0ED890E652D8B0E726E73291
:103EA000372F4CEF1FF00333023301330033362F2B
:103EB00046EF1FF0E750FF0FD8A00335D8B012002F
:103EC00029B18BEC1FF01200045100270551D8B026
:103ED000053D01270651D8B0063D02270751D8B04D
:103EE000073D032712000051086F0151096F02516D
:103EF0000A6F03510B6F12000101006B016B026B23
:103F0000036B12000101046B056B066B076B12005B
:103F10000335D8A012000351800B001F011F021FA0
:103F2000031F003F9BEF1FF0013F9BEF1FF0023F7D
:103F30009BEF1FF0032B342B032512000735D8A06D
:103F400012000751800B041F051F061F071F043FA7
:103F5000B1EF1FF0053FB1EF1FF0063FB1EF1FF0CB
:103F6000072B342B072512000037013702370337A0
:103F7000083709370A370B3712000101296B2A6B02
:103F80002B6B2C6B2D6B2E6B2F6B306B316B326B65
:103F9000336B120001012A510F0B2A6F2B510F0BAB
:103FA0002B6F2C510F0B2C6F2D510F0B2D6F2E5192
:103FB0000F0B2E6F2F510F0B2F6F30510F0B306FD8
:103FC00031510F0B316F32510F0B326F33510F0BD9
:103FD000336F12008984000EC76E220EC66E9E9645
:103FE000C69E000EC96EFF0E9EB602D0E82EFCD70C
:103FF0009E96C69E000EC96EFF0E9EB602D0E82E9B
:10400000FCD7C9CFABF59E96C69E000EC96EFF0EBB
:104010009EB602D0E82EFCD7C9CFACF59E96C69EC0
:10402000000EC96EFF0E9EB602D0E82EFCD7C9CF97
:10403000ADF59E96C69E000EC96EFF0E9EB602D0CE
:10404000E82EFCD7C9CFAEF59E96C69E000EC96E6F
:10405000FF0E9EB602D0E82EFCD7C9CFAFF59E96D4
:10406000C69E000EC96EFF0E9EB602D0E82EFCD78B
:10407000C9CFB0F59E96C69E000EC96EFF0E9EB6C5
:1040800002D0E82EFCD7C9CFB1F589949DEC22F07F
:1040900012008984000EC76E220EC66E9E96C69EC2
:1040A000800EC96EFF0E9EB602D0E82EFCD79E96FB
:1040B000C69EABC5C9FFFF0E9EB602D0E82EFCD748
:1040C0009E96C69EACC5C9FFFF0E9EB602D0E82ED6
:1040D000FCD79E96C69EADC5C9FFFF0E9EB602D008
:1040E000E82EFCD79E96C69EAEC5C9FFFF0E9EB6B3
:1040F00002D0E82EFCD79E96C69EAFC5C9FFFF0E24
:104100009EB602D0E82EFCD79E96C69EB0C5C9FFCB
:10411000FF0E9EB602D0E82EFCD79E96C69EB1C575
:10412000C9FFFF0E9EB602D0E82EFCD789949DEC05
:1041300022F012008984000EC76E220EC66E9E9673
:10414000C69E070EC96EFF0E9EB602D0E82EFCD7A3
:104150009E96C69E000EC96EFF0E9EB602D0E82E39
:10416000FCD7C9CFABF59E96C69E000EC96EFF0E5A
:104170009EB602D0E82EFCD7C9CFACF59E96C69E5F
:10418000000EC96EFF0E9EB602D0E82EFCD7C9CF36
:10419000ADF59E96C69E000EC96EFF0E9EB602D06D
:1041A000E82EFCD7C9CFAEF589949DEC22F0898426
:1041B000000EC76E220EC66E9E96C69E0F0EC96E6C
:1041C000FF0E9EB602D0E82EFCD79E96C69E000E2D
:1041D000C96EFF0E9EB602D0E82EFCD7C9CFB3F54C
:1041E00089949DEC22F012008984000EC76E220E85
:1041F000C66E9E96C69E870EC96EFF0E9EB602D0F4
:10420000E82EFCD79E96C69EABC5C9FFFF0E9EB694
:1042100002D0E82EFCD79E96C69EACC5C9FFFF0E05
:104220009EB602D0E82EFCD79E96C69EADC5C9FFAD
:10423000FF0E9EB602D0E82EFCD79E96C69EAEC557
:10424000C9FFFF0E9EB602D0E82EFCD789949DECE4
:1042500022F089849E96C69E8F0EC96EFF0E9EB672
:1042600002D0E82EFCD79E96C69EB3C5C9FFFF0EAE
:104270009EB602D0E82EFCD789949DEC22F0120065
:104280008984000EC76E220EC66E9E96C69E870E4D
:10429000C96EFF0E9EB602D0E82EFCD79E96C69E33
:1042A000000EC96EFF0E9EB602D0E82EFCD79E9679
:1042B000C69E800EC96EFF0E9EB602D0E82EFCD7B9
:1042C0009E96C69E800EC96EFF0E9EB602D0E82E48
:1042D000FCD79E96C69E800EC96EFF0E9EB602D07B
:1042E000E82EFCD789949DEC22F089849E96C69E88
:1042F0008F0EC96EFF0E9EB602D0E82EFCD79E969A
:10430000C69E010EC96EFF0E9EB602D0E82EFCD7E7
:1043100089949DEC22F012008984000EC76E220E53
:10432000C66E9E96C69E870EC96EFF0E9EB602D0C2
:10433000E82EFCD79E96C69E000EC96EFF0E9EB656
:1043400002D0E82EFCD79E96C69E000EC96EFF0EC8
:104350009EB602D0E82EFCD79E96C69E800EC96EF1
:10436000FF0E9EB602D0E82EFCD79E96C69E800E0B
:10437000C96EFF0E9EB602D0E82EFCD789949DEC44
:1043800022F089849E96C69E8F0EC96EFF0E9EB641
:1043900002D0E82EFCD79E96C69E010EC96EFF0E77
:1043A0009EB602D0E82EFCD789949DEC22F0120034
:1043B0008984000EC76E220EC66E9E96C69E8F0E14
:1043C000C96EFF0E9EB602D0E82EFCD79DEC22F0FF
:1043D0009E96C69E810EC96EFF0E9EB602D0E82E36
:1043E000FCD789949DEC22F08984000EC76E220EC2
:1043F000C66E9E96C69E8F0EC96EFF0E9EB602D0EA
:10440000E82EFCD79DEC22F09E96C69E010EC96E4A
:10441000FF0E9EB602D0E82EFCD789949DEC22F0C8
:1044200089849E96C69E910EC96EFF0E9EB602D0DE
:10443000E82EFCD79DEC22F09E96C69EA50EC96E76
:10444000FF0E9EB602D0E82EFCD789949DEC22F098
:1044500012008984000EC76E220EC66E9E96C69EFE
:104460008F0EC96EFF0E9EB602D0E82EFCD79DECD3
:1044700022F09E96C69E810EC96EFF0E9EB602D099
:10448000E82EFCD789949DEC22F012008984000E5E
:10449000C76E220EC66E9E96C69E8F0EC96EFF0E0A
:1044A0009EB602D0E82EFCD79DEC22F09E96C69ECA
:1044B000010EC96EFF0E9EB602D0E82EFCD789947D
:1044C0009DEC22F012008984000EC76E220EC66E8B
:1044D0009E96C69E910EC96EFF0E9EB602D0E82E25
:1044E000FCD79DEC22F09E96C69EA50EC96EFF0ECF
:1044F0009EB602D0E82EFCD789949DEC22F01200E3
:104500008984000EC76E220EC66E9E96C69E910EC0
:10451000C96EFF0E9EB602D0E82EFCD79DEC22F0AD
:104520009E96C69E000EC96EFF0E9EB602D0E82E65
:10453000FCD789949DEC22F01200050EE82EFED7E0
:1045400012000501256B266B276B286B899A400E9C
:10455000C76E200EC66E9E96C69E030EC96EFF0ED7
:104560009EB602D0E82EFCD79E96C69E27C5C9FFF0
:10457000FF0E9EB602D0E82EFCD79E96C69E26C59C
:10458000C9FFFF0E9EB602D0E82EFCD79E96C69EAF
:1045900025C5C9FFFF0E9EB602D0E82EFCD79E9619
:1045A000C69EC952FF0E9EB602D0E82EFCD7898A5D
:1045B0000F01C950FF0A01E1120005012E51130A33
:1045C00005E005012E51170A0CE012000501F00E5E
:1045D000256FFF0E266F0F0E276F000E286FFAEF64
:1045E00022F00501F00E256FFF0E266FFF0E276FDC
:1045F000000E286F899A400EC76E200EC66E9E96DA
:10460000C69E030EC96EFF0E9EB602D0E82EFCD7E2
:104610009E96C69E27C5C9FFFF0E9EB602D0E82E05
:10462000FCD79E96C69E26C5C9FFFF0E9EB602D039
:10463000E82EFCD79E96C69E25C5C9FFFF0E9EB6E6
:1046400002D0E82EFCD79E96C69EC952FF0E9EB69B
:1046500002D0E82EFCD7898A0F01C950FF0A1DE05D
:1046600005012E51130A05E005012E51170A0BE032
:1046700012000501000E256F000E266F100E276F29
:10468000000E286F12000501000E256F000E266F28
:10469000000E276F010E286F12000501256B266B97
:1046A000276B286B05012E51130A05E005012E51D9
:1046B000170A0CE012000501000E216F000E226F98
:1046C000040E236F000E246F6FEF23F00501000E20
:1046D000216F000E226F800E236F000E246F21C504
:1046E00000F122C501F123C502F124C503F125C55E
:1046F00004F126C505F127C506F128C507F1F2EC3E
:104700001CF000C125F501C126F502C127F503C142
:1047100028F5899A400EC76E200EC66E9E96C69EDC
:10472000030EC96EFF0E9EB602D0E82EFCD79E96F1
:10473000C69E27C5C9FFFF0E9EB602D0E82EFCD745
:104740009E96C69E26C5C9FFFF0E9EB602D0E82ED5
:10475000FCD79E96C69E25C5C9FFFF0E9EB602D009
:10476000E82EFCD79E96C69EC952FF0E9EB602D07A
:10477000E82EFCD7898AC950FF0A08E104C125F553
:1047800005C126F506C127F507C128F5D890050112
:1047900024332333223321332151F00B216F21673E
:1047A000D9EF23F02267D9EF23F02367D9EF23F065
:1047B00024676FEF23F00501100E2527E86A2623F2
:1047C000E86A2723E86A28231200E86A05012E51C7
:1047D000130A06E005012E51170A0BE0020E120023
:1047E00005012851000A03E12751F00B07E0010EF3
:1047F000120005012851000A01E0010E120029C52E
:1048000000F12AC501F12BC502F12CC503F125C524
:1048100004F126C505F127C506F128C507F181EC8D
:104820001EF003BF1200E5EC23F05FE1899A400E11
:10483000C76E200EC66E9E96C69E060EC96EFF0EF1
:104840009EB602D0E82EFCD7898A899A9E96C69E8B
:10485000020EC96EFF0E9EB602D0E82EFCD79E96C1
:10486000C69E27C5C9FFFF0E9EB602D0E82EFCD714
:104870009E96C69E26C5C9FFFF0E9EB602D0E82EA4
:10488000FCD79E96C69E25C5C9FFFF0E9EB602D0D8
:10489000E82EFCD79E96C69E000EC96EFF0E9EB6F1
:1048A00002D0E82EFCD7898A899A9E96C69E050E6C
:1048B000C96EFF0E9EB602D0E82EFCD79E96C69E0D
:1048C000C952FF0E9EB602D0E82EFCD7C9B05EEFEB
:1048D00024F0898A0501100E2527E86A2623E86A54
:1048E0002723E86A2823FFEF23F01200899A400E5D
:1048F000C76E200EC66E9E96C69E060EC96EFF0E31
:104900009EB602D0E82EFCD7898A899A9E96C69ECA
:10491000C70EC96EFF0E9EB602D0E82EFCD7898A5C
:104920000501256B266B276B286B1200899A400EB8
:10493000C76E200EC66E9E96C69E050EC96EFF0EF1
:104940009EB602D0E82EFCD79E96C69EC952FF0E98
:104950009EB602D0E82EFCD7C9CF33F5898A120063
:10496000899A400EC76E200EC66E9E96C69EB90EE0
:10497000C96EFF0E9EB602D0E82EFCD7898A1200BF
:10498000899A400EC76E200EC66E9E96C69EAB0ECE
:10499000C96EFF0E9EB602D0E82EFCD7898AFF0EA4
:1049A000E82EFED71200E5EC23F0D8A41200899A75
:1049B000400EC76E200EC66E9E96C69E030EC96E32
:1049C000FF0E9EB602D0E82EFCD79E96C69E27C547
:1049D000C9FFFF0E9EB602D0E82EFCD79E96C69E5B
:1049E00026C5C9FFFF0E9EB602D0E82EFCD79E96C4
:1049F000C69E25C5C9FFFF0E9EB602D0E82EFCD785
:104A00009E96C69EC952FF0E9EB602D0E82EFCD7D7
:104A1000898A0F01C950FF0AD8A4CEEF25F00501FD
:104A2000FE0E336FEAEC1FF0ABC534F5ACC535F5BF
:104A3000ADC536F5AEC537F5AFC538F5B0C539F5F6
:104A4000B1C53AF50784B6C166F1B7C167F1B8C11F
:104A500068F1B9C169F14BC14FF14CC150F14DC181
:104A600051F14EC152F157C159F158C15AF1F3EC0D
:104A700014F000C13BF501C13CF502C13DF503C195
:104A80003EF505015D674CEF25F05E674CEF25F0C4
:104A90005F674CEF25F0606750EF25F05DEF25F084
:104AA0005DC504F15EC505F15FC506F160C507F19E
:104AB00081EC1EF003BFCEEF25F059C13FF55AC17E
:104AC00040F5B5C541F5B6C542F507940501110E8F
:104AD000326F899A400EC76E200EC66E9E96C69E95
:104AE000060EC96EFF0E9EB602D0E82EFCD7898A4C
:104AF000899A9E96C69E020EC96EFF0E9EB602D081
:104B0000E82EFCD79E96C69E27C5C9FFFF0E9EB60F
:104B100002D0E82EFCD79E96C69E26C5C9FFFF0E82
:104B20009EB602D0E82EFCD79E96C69E25C5C9FF2C
:104B3000FF0E9EB602D0E82EFCD725EE33F0322FC2
:104B400002D0AEEF25F09E96C69EDECFC9FFFF0EC7
:104B50009EB602D0E82EFCD79FEF25F0898A899A6D
:104B60009E96C69E050EC96EFF0E9EB602D0E82E1A
:104B7000FCD79E96C69EC952FF0E9EB602D0E82E66
:104B8000FCD7C9B0B9EF25F0898A0501100E252799
:104B9000E86A2623E86A2723E86A2823120021C549
:104BA00000F122C501F123C502F124C503F1899A60
:104BB000400EC76E200EC66E9E96C69E0B0EC96E28
:104BC000FF0E9EB602D0E82EFCD79E96C69E02C16E
:104BD000C9FFFF0E9EB602D0E82EFCD79E96C69E59
:104BE00001C1C9FFFF0E9EB602D0E82EFCD79E96EB
:104BF000C69E00C1C9FFFF0E9EB602D0E82EFCD7AC
:104C00009E96C69EC952FF0E9EB602D0E82EFCD7D5
:104C100025EE33F00501100E326F9E96C69EC952E6
:104C2000FF0E9EB602D0E82EFCD7C9CFDEFF322F92
:104C30000DEF26F0898A1200899A400EC76E200E69
:104C4000C66E9E96C69E900EC96EFF0E9EB602D090
:104C5000E82EFCD79E96C69E000EC96EFF0E9EB62D
:104C600002D0E82EFCD79E96C69E000EC96EFF0E9F
:104C70009EB602D0E82EFCD79E96C69E000EC96E48
:104C8000FF0E9EB602D0E82EFCD79E96C69EC95255
:104C9000FF0E9EB602D0E82EFCD7C9CF2DF59E960A
:104CA000C69EC952FF0E9EB602D0E82EFCD7C9CFD1
:104CB0002EF5898A12006DEC1DF0B5C5E8FFD70806
:104CC00002E36DEC1DF0B5C5E8FFC80802E36DEC2A
:104CD0001DF0B5C5E8FFB90802E36DEC1DF0B5C5E0
:104CE000E8FFAA0802E36DEC1DF0B5C5E8FF9B08DC
:104CF00002E36DEC1DF09AEC20F0B0EC24F0F29C95
:104D0000F29E8B94C69AC2909482948C720ED36E4B
:104D1000D3A4FED789968A909390FF0EE8CF00F037
:104D2000E82EFED7002EFCD78150F294F29A9E9086
:104D30009D909E929D92F298F292F290F286F28E5F
:044D40000300FF006D
:10BF0000E844F926000C160C2B0C3F0C520C640C68
:10BF1000760C860C960CA50CB30CC10CCF0CDC0C6B
:06BF2000E80CF40C000C1B
:00000001FF
